:020000040000fa
:080000000004040000000000f0
:020000040000fa
:100800006f9e2000807f240000018800000000000f
:100810000a00070011000700000020000000e000af
:10082000020032000000020000000000240f02005d
:10083000000000000040da000000fe004440a90073
:10084000001820000000e00003003200000020003b
:10085000a00188004440a80000000600000221001a
:10086000010020001600370062004000e0804800d0
:10087000910188009001ba0062004000e0804800c9
:10088000910188009002ba0062004000e0804800b8
:100890000002eb006028e10005003a008301e90056
:1008a00007003300038009000059eb000400370003
:1008b0006128e100010032000082eb000500070022
:1008c000910188001001ba000200e000e6ff3a0042
:1008d000000005009101880080027800620040005d
:1008e000e08048003559ba008301e9000800320071
:1008f0002559ba008301e900050032000400e00038
:10090000f4ff320015d9ba008301e900f1ff3a0083
:0409100000000600dd
:020000040000fa
:020000040005f5
:0457f400ffff0000b3
:020000040000fa
:020000040005f5
:0457f800be130000dc
:020000040000fa
:020000040005f5
:0457fc007f3e0000ec
:020000040000fa
:100008004a1000004a1000004a1000004a10000080
:100018004a1000004a1000004a1000004a10000070
:100028004a1000004a1000004a1000004a10000060
:100038004a1000004a1000004a1000004a10000050
:020000040000fa
:020000040000fa
:10280000c0f72f004027b6000004040000000000bd
:0428100000000600be
:020000040000fa
:100914000a850000d6840000b08400000e85000023
:1009240006000000ff09000001a1000001190000f9
:10093400012900004015000000260000ff0000000f
:1009440075080000954000008102000019010000b4
:100954002940000091020000c000000026030000ae
:100964005500000053000000420000002000000079
:10097400480000004900000044000000200000007e
:10098400420000006f0000006f00000074000000cf
:100994006c0000006f0000006100000064000000b3
:1009a4006500000072000000340300004d000000e8
:1009b4006900000063000000720000006f00000086
:1009c400630000006800000069000000700000007f
:1009d40020000000540000006500000063000000d7
:1009e400680000006e0000006f0000006c00000052
:1009f4006f00000067000000790000002000000084
:100a0400490000006e000000630000002e0000009a
:100a1400040300000904000009020000290000008a
:100a24000101000000c000003209000004000000c1
:100a34000002000003000000000000000921000083
:100a44001101000000010000221d00000007000049
:100a540005810000034000000001000007050000bc
:100a6400010300004000000001000000120100002a
:100a7400100100000000000000080000d80400007d
:100a84003c00000002000000010200000001000020
:020000040000fa
:100a94008180fb00120020000111dd000248780073
:100aa4000000060010478000104278008480fb009c
:100ab40070478000808f50000300360000427800a9
:100ac4008441780009003700010050007047880015
:100ad400fbff3700504780000381fb008197200013
:100ae40062d87800504788008341e9000304e0009d
:100af400f8ff3a0001478000ee08e2000e003200e1
:100b040080c0b300804878000147800080972000af
:100b14009000980010478000104090000068a300e7
:100b240002003a0080ccb3000100370080c8b30053
:100b34009040980000000600009820009000980063
:100b4400ece8a90000000600a08d200021c0b3003d
:100b540090cf10001a003a0094c4bf000058a300bc
:100b6400170032001047800081c0b30090cf1000fe
:100b740013003a0010409000c043b20041c3b300d8
:100b8400814f50000e003a00014780001140900050
:100b94000004e0000a00350000982000900098004e
:100ba4000001eb008197200000982000617079001b
:100bb4000201e800e80f510010003200f9ff37008d
:100bc4000041eb0002007800dae8b70081c0b3000e
:100bd4000047800001487800014780000098200009
:100be40090009800c0c8b30090409800304780003f
:100bf4001240980030478000124098000000060020
:100c0400a08d200021c0b30090cf100001003a0055
:100c1400a4ff3700ccff3700a047800083002000ea
:100c2400e70f500009003e0080017800dbc8bf00d8
:100c340002003a0010c0b30003003700e14f500037
:100c440002003a0020c0b300dbe8b700324780005e
:100c540012409000c818de00014070001041980056
:100c6400304780000348780003007800f428b5007a
:100c740080972000c0468800904780006100600093
:100c84000001eb0011003a00000178000600370073
:100c9400c04680008147800031587800c0468800f3
:100ca400814788000201e800830f5100f8ff3a00f1
:100cb40000000600c046800081478000315878005b
:100cc400c0468800814788000201e800830f510074
:100cd400f8ff3a0000000600889fbe000998200033
:100ce40094a4a900f2e8ab0009003a0081c0b30063
:100cf400004780000148780001478000990098006f
:100d0400c0c8b3009040980041c8b3001c0037002d
:100d140080c9bf0008c8b300884060001b003200cf
:100d2400314c8000a0478000808f500002003100c9
:100d3400304c8000a0478800b7ff070010c0b30004
:100d4400dae8b70081c0b3000047800001487800aa
:100d54000047800019009800184098001047800050
:100d64000148780010478000190098001840980046
:100d740081972000304780001100980081ccb30097
:100d840030478000114098000e00370020c0b300a7
:100d9400dae8b700304780000148780082ccb3001d
:100da400304780001240980081c0b30000478000a3
:100db4000148780001478000809720009000980047
:100dc400924098004f04be0000000600881f78007f
:100dd40030478000104090004600de00610460004f
:100de400708f200081c0b30090cf100008003a003b
:100df40082c9bf000080fb00b024880000c1b3009a
:100e04009604e20001003a0040c0b300f7e8b700de
:100e1400a08d200011c0b30090cf100013003a0041
:100e24008097200031478000900098007aff0700e7
:100e3400b08d200021c0b30090cf100004003a0010
:100e440041c8b300304780001140980008003700c3
:100e54003147800080ccb3000804e0000100320078
:100e640080c8b300904098000100370036ff0700a7
:100e74004f0478000000060001982000914078009b
:100e840000c8b30080cf50001f003a0000ccb3006c
:100e9400f2e8b70083c9bf00e24f500008003200f7
:100ea400e34f50000e003200e14f500015003a00ad
:100eb4008053280080478800200120000f0037005d
:100ec40082c9bf000080fb000000400001492800e7
:100ed400e080780081478800110090000700370007
:100ee40082c9bf000080fb0000004000a148280028
:100ef40060807800804788001080fb00a04788004d
:100f040000000600f268ef00000006007869ef00b8
:100f14007969ef0000982000104078007f4060005d
:100f24000080fb00e10f50000b003200e20f500084
:100f34000b0032000000e0001a003a00f2e8a800ba
:100f44007809a800b0468000e10f500015003a006f
:100f54007829a80013003700f2e8a8001100370030
:100f6400f2e8a80084c9bf004198200091407800ad
:100f74008180fb006f006000c708de0000004000b5
:100f8400010040004200dd0001802000010040001b
:100f9400104090000028a3000200320010c0b300eb
:100fa40078e9b700f2e8ab00050032008097200032
:100fb40080478800f208a80020c0b300f4e8b70016
:100fc4000000060082c9bf00e14f50000b003a0048
:100fd40080c9bf007f40600008003a00f2e8a80022
:100fe40081c9bf00e34f500003003a001000200005
:100ff400b046880001003700d628ef008249e2009d
:1010040026003a0080c9bf00ff406000e2cf5000d4
:1010140022003a0084c9bf006f4060001f00320004
:10102400f2e8a8008141780084c9bf0041982000fb
:10103400914078008180fb006f0060000000400058
:10104400c708de00010040004200dd0001802000ee
:101054000101400081c9bf00e34f500002003a0083
:1010640040c8b3000a00370084c9bf006f006000a5
:1010740000004000a14a2000010040001010a1001f
:1010840000c4b3008449e2000100350080ccb30001
:10109400104198008341e900e3ff3a000000060094
:1010a400f2e8a800e468ef0082c9bf00f6e8b700e0
:1010b4008249e20003003a0000c1b300f7e8b70038
:1010c4000000060000c2b300f7e8b700730337005e
:1010d40080c9bf000046b20030003a0081c9bf0099
:1010e4000080fb0001002000eb0f5000e08f58004f
:1010f4002a003e000060010013003700130037008f
:10110400260037001100370024003700060037009e
:1011140009003700200037000900370007003700b6
:101124000b00370014003700f2e8a80080c0b300b9
:10113400f7e8b700000006004fff3700d8ff37007c
:10114400608f20000600370070ff37009dff3700d6
:1011540084c9bf000080fb00418e200001004000d4
:1011640080478800f208a80010c0b300f4e8b70074
:10117400f2e8a80000000600f2e8a80084c9bf0055
:101184000080fb00418e200022982000124178004c
:1011940002f07800000006003f030700000006008c
:1011a40031478000114090000004e00002003d003f
:1011b4000040eb0090409800db68ef00da68ef0035
:1011c400f428ef00f268ef00c1ff070031030700c5
:1011d400c1fe3700d4c8bf008080fb000100780046
:1011e4000020a1000000e0000c003a00c10fb20092
:1011f40000802000008040001047880000478800dd
:1012040010409000c043b20041c3b300814f50006e
:1012140001003a00e2ff370079fe3700e80f500082
:1012240001003a00e9fe0700000006000080fb0010
:10123400800140000180fb00008041004200dd008d
:101244000280200002014000124090000070a100c2
:1012540010419800c08d20000104e000010032001c
:10126400608e200082317800124090000060a0005f
:101274001041980000000600889fbe00804478005a
:101284000184fb000080fb0000004000a14a200014
:1012940008b078000838a300030032008040eb0057
:1012a40009407800e1ff07000828a300030032008a
:1012b40011c0b30009407800dcff07004f04be00f2
:1012c400000006000080fb00000040008180fb005d
:1012d400010040004200dd000180200001004000c8
:1012e4009040900042c8b30082c070001140980042
:1012f400000006000080fb000104e000030032004f
:1013040080004000608e2000020037008000400012
:10131400c08d200061027800144090000064a20097
:101324001042980012029800034a7800144090007a
:101334000044b200104298001440900081c8b300e9
:10134400014070001042980004007800000006007c
:10135400f00f20007024880050248800f009200039
:1013640080248800b00f2000602488008804a8002e
:10137400018020004808de00c02488009424a800ce
:101384009424a9009624ef000000eb008018eb00e1
:101394008018eb000000e800e40f5000fbff3a0067
:1013a400d0002000502588000200370080c0b30020
:1013b4008ae4b7008ac4bf000038a300fbff3a00e8
:1013c40021c0b3008140e900feff3a00010078002b
:1013d400f2e8b70094a4a9004080200030478800b8
:1013e4008000fd00f6e8b700f7e8b7008000fd00d4
:1013f40000000600aac4bf000018a3000d003200bc
:10140400124780009240900000c8b30080cf500083
:1014140007003a00304780009040900040c8b30075
:1014240080cf500002003a0068404000104198000c
:10143400aa24a90040c0b3008ae4b7000000060053
:101444008284a80000c1b3008ae4b7008d0237008b
:101454008d0207008284a90000c1b30080e4b700b4
:1014640000000600881f7800f748e2000c003a00ec
:101474009424ef008c24ef00010037009404a800aa
:1014840094c4bf000008a300fcff320010c0b300e6
:10149400f7e8b700a624ef000001200040258800eb
:1014a400708f200011c0b30090cf100007003a00e5
:1014b400f00f2000502488008c24ef008c04a80036
:1014c4008c84a80020c0b300f7e8b70080c4bf0034
:1014d4000048a3000400320082c4bf000048a300f7
:1014e40001003200daff070088c4bf000018a3001f
:1014f40041003a008ac4bf000008a3000e00320075
:101504008cc4bf000008a3000b00320090ff07004a
:1015140040c0b300f7e8b7000098200010408800ee
:1015240080c0b30000e8b70030c0b3000168b60063
:10153400c0c8b3000168b7008ac4bf000048a30054
:10154400040032008cc4bf000048a3000100320034
:10155400bbff07008ac4bf000028a30006003200b6
:101564008cc4bf000028a300030032004702070018
:1015740040c0b3008ae4b7008a44e20003003d009f
:101584008c44e20001003d009aff07008ac4bf00ba
:101594000018a300060032008cc4bf000018a3008a
:1015a400030032003a020700f00f20007024880084
:1015b400708f200031c0b30090cf10000e003600b1
:1015c4008cc4bf000038a3000b00320048c0b30035
:1015d4008ac4bf000038a3000700320090248000b2
:1015e400d4e8b70080c0b3008ae4b700f9fe07006e
:1015f4000844e900f6ff3a004f04780000000600b2
:10160400201680008000eb002116880000f02f00d7
:10161400c022b600d8c2a800d8e2a800014f8800b2
:10162400f14e880012002000e24e880090cab300f8
:10163400dae9b70000802a00b04e880020002000bc
:10164400c04e8800020078008ce9b70001007800e1
:10165400d5e9b7008ea9ef0090a9ef00010078004a
:1016640092e9b700000006008809e20002003a008f
:1016740000712200404c8800424c80000201e900c5
:10168400424c880088c4bf000018a3001300320035
:101694000200e00049003a00412c2000914078000b
:1016a4000104a200e1c06000c4c2bf000004a100a4
:1016b40001407000c4e2b700412c20009140780042
:1016c400e1c0600081c04000c4c2bf000014a1009a
:1016d40001407000c4e2b70000000600718f2000d2
:1016e400914078000104e00002003a00c402a9001d
:1016f40019003700e1cf500002003a00c402a800ec
:1017040007003700e2cf500002003a00c402a800ec
:1017140011003700e4cf500003003a00c402a900ce
:10172400c422a80000000600f0cf50000c003a00cc
:101734000200e00021003a00412c20009140780092
:101744000104a200e1c06000c4c2bf000004a10003
:1017540001407000c4e2b700c422a90000000600e2
:1017640000c2b30080cf500014003a000200e00031
:1017740012003a00412c2000914078000104a2009c
:10178400e1c06000c4c2bf000004a10001407000b9
:10179400c4e2b700c4c2bf000004a20061406000fc
:1017a40000404000412c2000914078000114a10029
:1017b40080c0700001007800c4e2b7000000060099
:1017c400d4c9bf000080fb00010020004a09dd00ed
:1017d400c600de00810071004a00dd0022042400fe
:1017e400023b88000181fb00920188000081eb002c
:1017f4000208bb001000fc0050052000303b8800ac
:10180400a00a2000303b880061e7a8000000000027
:10181400000000006147e200feff35000000060002
:1018240030002400003b8800449920001600370053
:101834000080fb0001002000724c8000834c80007b
:101844000001510081815900930188001409bb00f3
:10185400140090000089bb001000fc005505200016
:10186400353b8800a50a2000353b880061e7a800c5
:1018740000000000000000006147e200feff3500a8
:1018840092e9ed006402420092c9bf00e8ff3a0009
:1018940061c7a900000006000400fa00e0bf9f0031
:1018a400f1bf9f00910180007fb8970090018800ec
:1018b4006fb897009081ba001001ba0091018800b6
:1018c4000200be000080fa0000000600881f7800b5
:1018d400d549e2001b003a00004f80000000e00000
:1018e40003003200104090000004e000470135007e
:1018f4008000eb00028120000089200062f0780063
:101904008100e80000042000808f5000f9ff3a00b5
:10191400814178008040eb0010c0b30075fe0700e1
:10192400004f880010c0b300d5e9b700018520003e
:101934008058eb0000892000808f50003301320072
:10194400fbff37000389200093417800e5cf510065
:101954008100320006003e00e3cf51004d0032000a
:101964005f003e00e2cf510028013a000600370034
:10197400e7cf5100ca003200c5003900e8cf51005a
:1019840022013a001a0137000300780050e8b7003a
:1019940080c3b30051e8b7000300780052e8b700f1
:1019a40014c0b3000400780053e8b7005468ef0093
:1019b40040c1b30055e8b7005668ef005768ef0020
:1019c40000c02e00f1ff2f00b64e8000c74e8000ed
:1019d400060040008780480058e8b7004801de0050
:1019e4000200780059e8b700010078005ae8b7000f
:1019f4004808de005be8b7005ce8ef008c49e200d1
:101a04001a003a00040078005ce8b7005d68ef0053
:101a14005e68ef005f68ef006068ef006168ef00e8
:101a240040c0b30062e8b7006368ef006468ef0089
:101a340030c0b30065e8b70080cfb30066e8b700f4
:101a4400b0cab30067e8b7000300780068e8b700dd
:101a54006968ef0080c0b3006ae8b7006b68ef0004
:101a64006c68ef006d68ef006ee8ef00f04e8000e8
:101a74000000e00003003200104090000004e00089
:101a8400e200350003c4b3000285200084407800de
:101a9400d20037009148e20008003a00a0cab3001f
:101aa400dae9b70087bf2a00b74e88002700200074
:101ab400c74e88008c69ef00cb00370090cab30092
:101ac400dae9b70000802a00b04e88002000200028
:101ad400c04e880010c0b3008ce9b700c2003700c4
:101ae40050c0b300d4e9b7000300370034ff070047
:101af4005cfe0700d469ec00419d20009140780011
:101b04008180fb00dac9bf000080fb000000e80010
:101b1400808f5000f5ff35008c49e2000c003a003c
:101b24008000eb00910188000080eb008008bb007e
:101b34000c00fc0058052000383b8800a80a20004f
:101b4400383b880061e7a8000000000000000000a6
:101b540061c7a900a4003700704c8000814c80004c
:101b6400e10f4000e08f48000e003a001189200088
:101b7400914078008180fb0092c8bf004800dd00de
:101b84000101700031892000914078008180fb00c0
:101b940094c8bf004800dd0081017000724c8800c9
:101ba400834c880011892000914078008180fb00db
:101bb40092c8bf004800dd00010170003189200097
:101bc400914078008180fb0094c8bf004800dd008c
:101bd400810170000004eb00704c8000814c800097
:101be400820f5000838f5800220032007e0037009d
:101bf40024992000144278008481fb0083814100f1
:101c04008003200001005000220020001100090080
:101c14000200d8008580fb00010040000000400065
:101c240081892000010040009080fb00104090005a
:101c34004800dd00010070004199200080b1780067
:101c44000442e8000400780092e9b700764c800072
:101c5400874c800061034300e0834b00764c88008e
:101c6400874c8800fc4f520001003a00ecfe07004c
:101c74000804e8008842780095c8bf008080fb0013
:101c84000100d100804f5400d9ff390056003700bd
:101c9400e3fe07008ea9ef0090a9ef005200370081
:101ca4000300780050e8b7001189200091407800c3
:101cb4008180fb0092c8bf004800dd000101700074
:101cc40031892000914078008180fb0094c8bf00d6
:101cd4004800dd00810170000200780051e8b7007f
:101ce4004810de0052e8b7000300780053e8b7005c
:101cf4004818de0054e8b70095c8bf0055e8b7009f
:101d04000044eb002700370013892000934178003a
:101d14008381fb0022892000124178004811dd00f4
:101d24000300710033892000934178008381fb0014
:101d340042892000124178004811dd0083007100bf
:101d44000881fb000300200000004100818049005d
:101d5400d1fe07008881fb005289200012417800df
:101d64000281fb000201d100828151008381410084
:101d74000289200002814100004978004802de0007
:101d84001441980081037800f70fb20020892000e5
:101d940080814100874978004838de0090419800ee
:101da40008c4e80095c8bf000080fb000000d10013
:101db400804f5400d4ff3900f04e80000000e00052
:101dc40003003200104090000004e0000f003500d2
:101dd40003c4b3000285200011c0b30001407800a1
:101de40044fd0700f04e8800d569ef000700370076
:101df4009424ef000000eb00000000000000e80065
:101e0400e10f4000fcff3a000000fe004f047800a0
:101e140000000600dc09e2000100320012fe0700a7
:101e2400708f2000f1c1b30090cf10000400360081
:101e340088c4bf000018a30001003a00a3fe0700f5
:101e440000000600d8c2a800dac2bf000068a300e0
:101e540005003200003a80003008b200020032006f
:101e640000140400000000002ca3ef0038fd07005c
:101e7400e3fd0700c422ef007afd0700e5ff070039
:101e8400fdff370000000600000006000000060009
:101e9400000006001900370000000600d1c1b3009d
:101ea40010c0b300f4fc070003c4b3000281200097
:101eb4008040eb0010c0b3000efd0700004f880007
:101ec400000006009444a80080702000504c880054
:101ed4008000eb008100e80080702000808f5000bb
:101ee400fcff3a008a29ef009444a9000000060090
:101ef40000000600000006000000060080c9bf00c4
:101f04007f406000e14f50004b003a008449e200fa
:101f140049003a0081c9bf00e64f50001f003a0053
:101f240031982000914078007c40400080cf5000e0
:101f34000e0032000040e80080cf5000150032004f
:101f440000c0e90080cf500014003a00608f2000e8
:101f540011c0b30090cf100010003a0000522800c6
:101f6400804788009000200007003700608f200021
:101f740011c0b30090cf100008003a002049280097
:101f840080478800d0012000a047880000ccb3001f
:101f94000100370000c8b300f2e8b70080c9bf00f1
:101fa4000046b20001c2b300814f500022003a0043
:101fb40081c9bf00e34f50001400320003003e000b
:101fc400e24f50001c003a0005003700ea4f500071
:101fd40009003200eb4f500017003a00120037009e
:101fe400309e20008047880010002000a047880011
:101ff40010ccb3000a00370000c8b300f2e8b70001
:1020040083c9bf00e3e9b70000000600209e20005a
:102014008047880010002000a047880010c8b30043
:10202400f2e8b7000000060000c8b300f2e8b70009
:0c20340082c9bf00e2e9b700000006000e
:020000040000fa
:10204000dc090000060000000200000001000000a2
:10205000000000008809000054000000000000009b
:1020600010080000c000000000000000e2090000ad
:102070000400000000000000d0080000b8000000cc
:102080000000000000080000100000000000000038
:04209000000000004c
:020000040000fa
:042094000000fe004a
:00000001FF
